:020000040000FA
:100000004028000000000000A000030E8312A100A1
:10001000E022210E8300A00E200E09007F39CE229F
:10002000031C0F2808008401A001840B1528A00BD5
:100030001528FF3E0318152808008B138B120B118F
:100040000710031496220130132087160310D321C2
:1000500003102C21053013200B108B1563008B111E
:100060000B100314D32103102C210430132087120A
:100070008B168B17FF30A6000130D523080008002F
:100080002030840040308001840AFF3E031D432855
:10009000073099008316FF2390003F3085001C3005
:1000A00087000830810007309500303096008312B9
:1000B000C822B02020213130900003102C210130C3
:1000C000D5238B1787120F0822060319AD28A20625
:1000D000803903196E28A408031DA403A30D23105F
:1000E00085192314A50D251005192514A60D261014
:1000F000851A2614271882282508031D8528271409
:100100006F218528250903192710A7188F28230890
:10011000031DA728A71427110830A400A728240826
:10012000031D9B2827199B282715031496220330AB
:10013000A2210830D5232309031DA728A7100310E7
:1001400096222719A7280330BE210930D523260877
:10015000031DAD281D20FF30A6003323DB216328BB
:100160008316051485148510831285100000000085
:1001700083160510831205100000000083168514F5
:100180000000000005148312080083168514000087
:10019000000005148312051CCB28031085180314D6
:1001A0008316051083120800A8000830A80D8316D6
:1001B00003188514031C8510000000000514831229
:1001C000051CE0280000831605108312FF3E031D66
:1001D000D628C5200800831685100000051083125C
:1001E000D4200800831685100000000005140000CC
:1001F0000000851483120800A8008316851483125A
:100200000830A900831605148312051C0529000077
:10021000031085180314A80D831605108312A90B6B
:1002200002298316031C85100318851405148312F4
:10023000051C1829000083160510831228080800E1
:100240000130AA002030B100DC30AF002E30B00009
:100250000030BE21871008002A1203182A168714BE
:100260000A30B700B70B3229C030EB2003185129F0
:1002700030083F392A1940382A11AA188038D4206A
:100280002A1A51292F08D42031088038AA19103889
:10029000AA1E0138D4201A302A1CC038D42040307D
:1002A000D420F2208710080087140A30B700B70B5B
:1002B0005729C130EB2003186C290301FC20B20040
:1002C0000301FC20B3000301FC20B4000301FC2067
:1002D000B5000130FC20B600F220871008002B1476
:1002E000AB10080084003A08031D862900086E3E02
:1002F000AF00840A00080318013EB000AA150310DD
:100300002C210F08103EAD000430BA000800840014
:100310000301AA1937302F028000840A3008031C19
:10032000FF3E8000080084003A08031D9A29031448
:100330002C21542134088000840A3508F039033810
:1003400080000800B7000310DF2303140301DF233C
:10035000B70A37080310DF2303142F08DF23370AF7
:100360000310DF2303143008AA198038DF23370372
:100370000310DF230314C530DF230800B700D723A1
:10038000C53A031DD229B70A3708D723AF00370A69
:10039000D723B700AA11B71BAA157F39B000AA103E
:1003A00003102C2108002A140318DA292A10AA1293
:1003B0000030A22108002B1DE2292B11BA01AA103E
:1003C000AA12932AAB110F082D028039031DAB1519
:1003D00001308A003A088207F229282A442A542A3E
:1003E000732A812A2B180A2AAB1D952AAE0A2E08D9
:1003F000043C0318FC29AE010F08323EAD00AA1FD1
:10040000042A5421AA132A132A1F952A03142C21E3
:10041000AA17952A2B10AA1D112A3730AF02031CE8
:10042000B003AA110C30AF070318B00AA0222F089E
:10043000693C3008031C013E333C0318232A9E30DC
:10044000AF002930B000AA142A15AA16BA0A932AB6
:10045000AB1D952A5421B21F402A3308AF00320841
:100460003F39B000321F3F2ABA01AB183A2AAB1409
:100470002B14952AAA10AA120130D523932ABA0A5E
:100480000F080B3EAD00952AAB1D952A5421350E61
:100490000F39AC00AA153730AF070318B00A0F08A0
:1004A000103EAD00BA0A932AAB1D952A5421350E91
:1004B0000F392C02031C003C013C031C702A340839
:1004C0007F39313C0318702A0D3E031C702A3730E7
:1004D000AF070318B00A0F08103EAD00BA0A932AFE
:1004E0002B14BA01952AAB1D952A54213508AC006E
:1004F0006E30AF02031CB003BA0A0F08063EAD000F
:10050000932AAB1D952A5421AA10AA12BA013508C4
:100510002C020318902A3730AF070318B00A912A2B
:10052000AA110130D52303102C210800AA120318A8
:10053000AA1603102C2108000310AA1A031408009D
:100540002F08B7003008B8009230B702031CB80378
:100550002930B8020930B9000630B7020318B42AAE
:1005600038080319BB2AB803B90BAC2A0130B7020B
:10057000031CB803AA2A0330B7073707AF02031CCE
:10058000B003B71BC72A0630AF070318B00A08002C
:100590000730C90007100B118B1608000310BB1899
:1005A000D42ABE00BB14031408000310BB1C0314A0
:1005B00008000310C11DDF2A0314C11144080800FC
:1005C0000B11A83081000508C6003B18F82A3B1D16
:1005D000EC2A3B113F08F02ABB1C052BBB103E0840
:1005E000BC0007140A30BD000430C0003B14052BCA
:1005F000C00B052B0314BC0C031C071403180710B5
:100600000430C000BD0B052B3B10071E0B2B4718F9
:10061000192B47140D2B4710192B0310071903141E
:10062000C80CC90B192B0314480CBF003B1507302D
:10063000C900411D2B2BC50B322BC30B242B4208A9
:10064000C400C1154111322B0310461E0314C20C05
:100650000430C500322B461E322B0530C500093050
:10066000C30041150800D922031C8D2BCB001B3A77
:100670000319CA0103308A004A088207452B4A2B16
:100680007A2B7A2B7A2B7A2B842B1B304B0603196F
:10069000CA0A8D2BCC01CD01CE01CA0151304B06C7
:1006A0000319672B52304B0603196B2B4D304B0649
:1006B00003196E2B4E304B060319722B53304B0629
:1006C0000319762B58304B060319782B8D2B0230EB
:1006D000CA004E148D2BD1142A178D2BAA14031483
:1006E0002C218D2BAA1003142C218D2B1D208D2B3A
:1006F0006F218D2B0430CF00CB0ECB0DCC0DCD0D4B
:10070000CF0B7D2BCA0A8D2B4D0A03198A2B4C3037
:1007100072218C2B0130D523CA01D522031CD42B86
:1007200003308A00500882079D2BB22BB72BBC2BBD
:10073000C52BC52BC52BC52BD22B5118A62BD11CD5
:10074000A32B2A1FA92BD119AC2BD42B0130D000FD
:10075000AF2B0230D000AF2B0330D000AF2B1B30BB
:10076000CE22D42B5110523087215130C12BD110C1
:10077000523093215230C12BD11152308721563043
:10078000C12BCE220430D000D42BCF010430D20DA7
:10079000D30DCF0DFF3E031DC72B30304F07CE22A8
:1007A000D00AD42BD001D42B0800D1040800831622
:1007B0009C18D82B9B001C141A088312080083165F
:1007C000031C9B0003189A00031CF42B1C158B13AD
:1007D00055309D00AA309D009C148B179C18EE2B61
:0C07E0001C1103109C1D03148312080060
:084000000200080000000900A5
:02400E00C411DB
:00000001FF
